S01100004C43444D61747269782E73726563CB
S113000045C000004BC0000049C0000047C00000CC
S113001045C0000043C0000041C000003FC00000D4
S11300203DC000003BC0000039C0000037C00000E4
S113003035C0000033C0000031C000002FC00000F4
S11300402DC000002BC0000029C0000027C0000004
S113005025C0000023C0000021C000001FC0000014
S11300601DC000001BC0000019C0000017C0000024
S113007015C0000013C0000011C000000FC0000034
S11300800DC000000BC0000009C0000011241FBEF9
S1130090CFEFD0E1DEBFCDBF41D06EC0B1CF109263
S11300A0710080E280937000089584EA8093740064
S11300B0809174008823E4F7089584E980937400A0
S11300C008958093730084E8809374008091740091
S11300D08823E4F7089520E030E008C0E3ECF9E079
S11300E03197F1F700C000002F5F3F4F2817390701
S11300F0ACF30895CF93DF93D8DF80EEE2DF80E0A6
S1130100E0DFC0E0D0E003C080E0DBDF2196C03157
S1130110D105D4F3D2DFDF91CF910895C0DFC5DFDD
S113012080EECFDF81E2CDDFC8DFBFDF80EEC9DF45
S113013080EAC7DFC2DFB9DF80EEC3DF83EEC1DF51
S1130140BCDFB3DF80EEBDDF81E8BBDFB6DFD2DF2B
S1130150C0E0D0E00CC0A9DF80EEB3DF8C2FB1DFAC
S11301608FEFAFDFAADF88EC90E0B5DF2296C031D5
S10F0170D1058CF3BFDFECCFF894FFCF77
S9030000FC
